:100000008228A4008417800484138E010C1C8E00A7
:10001000222003197D28222003197D282228A400EC
:1000200031200C080D0403197D287720841324083F
:10003000800664001B281C288C0A03198D0F1928C0
:1000400080067D2824088E0601308C008D01000872
:1000500024050E06031D08008C0A03198D0F27289E
:100060000800FF3A841780057D288F018E00FF303D
:100070008E07031C8F07031C7D2803308D00DF30A3
:10008000432037288D01E83E8C008D09FC30031C8D
:100090004C288C07031849288C0764008D0F4928C9
:1000A0000C1852288C1C56280000562808008E0078
:1000B000033060288E00013060288E0006306028F2
:1000C00094000F080D02031D67280E080C0204306F
:1000D00003180130031902301405031DFF307D2879
:1000E0000038031DFF300405031DFF307D288C09F7
:1000F0008D098C0A03198D0A0800831303138312D8
:100100006400080083160830850086018312F328F6
:1001100001308C0005308400083001200C08B0004C
:100120000D08B10030088C0031088D008F0150306F
:100130005720031D9D28B701080030088C003108A6
:100140008D008F017A305720031DA9280130B70098
:10015000080030088C0031088D008F018E30572048
:10016000031DB5280230B700080030088C003108A4
:100170008D008F01A2305720031DC1280330B70026
:10018000080030088C0031088D008F01B6305720F0
:10019000031DCD280430B70008000530B700080063
:1001A00028088C0029088D000630840001300F20BB
:1001B0002A088C002B088D000630840002300F20A6
:1001C0002C088C002D088D000630840004300F2090
:1001D0002E088C002F088D000630840008300F2078
:1001E0000A30352008005C30A800A901D430AA00EC
:1001F000AB01D430AC00AD015C30AE00AF01D0201B
:10020000882028088C0029088D008F015C305D2033
:100210009E002C088C002D088D008F01D4305720B3
:10022000A0001E08840020087020A000A100640027
:100230002008210403191D29B50128088C0029086C
:100240008D008F015C305D209E002C088C002D08F5
:100250008D008F015C305D20A0001E088400200806
:100260007020A000A10064002008210403193A298D
:100270000130B50028088C0029088D008F01D4308A
:1002800057209E002C088C002D088D008F01D43043
:100290005720A0001E08840020087020A000A100A4
:1002A000640020082104031957290230B5002808EA
:1002B0008C0029088D008F01D43057209E002C0817
:1002C0008C002D088D008F015C305D20A0001E0881
:1002D000840020087020A000A100640020082104F0
:1002E000031974290330B5003708053C031C822923
:1002F00001308A0037088207B12B83298F29AB2967
:10030000C7298329FF283508033C031C8F290130A6
:100310008A0035088207A32AE329432AFF280130EF
:10032000B4006400C930340203189929D020B40FF6
:100330009129882064003708023C031DFF283508F6
:10034000033C031CAB2901308A0035088207432A8D
:10035000FF28272B102A0130B4006400C930340272
:100360000318B529D020B40FAD29882064003708C0
:10037000033C031DFF283508033C031CC72901303B
:100380008A0035088207FF28702A102AE52A0130E2
:10039000B4006400C93034020318D129D020B40F4E
:1003A000C929882064003708043C031DFF2835084C
:1003B000033C031CE32901308A0035088207E32946
:1003C0006C2BFF28702A0130B200B30132088C0078
:1003D00033088D008F0178305A20031D0F2AA80A98
:1003E0000319A90A32088C0033088D008F011E30D2
:1003F0005D20031D012A0130AA020030031C013ECA
:10040000AB020130B40064000630340203180B2A3A
:10041000D020B40F032AB20A0319B30FE629FF282C
:100420000130B200B30132088C0033088D008F0117
:1004300078305A20031D3C2A0130A8020030031CEA
:10044000013EA90232088C0033088D008F015A301A
:100450005A20031D2E2AAA0A0319AB0A0130B40040
:100460006400063034020318382AD020B40F302A32
:10047000B20A0319B30F132A5C30A800A901D430C3
:10048000AA00AB01FF280130B200B30132088C0092
:1004900033088D008F0178305A20031D6F2A0130F8
:1004A000AC020030031C013EAD0232088C00330860
:1004B0008D008F011E305D20031D612AAE0A0319D5
:1004C000AF0A0130B40064000630340203186B2A0E
:1004D000D020B40F632AB20A0319B30F462AFF28AB
:1004E0000130B200B30132088C0033088D008F0157
:1004F00078305A20031D9C2AAC0A0319AD0A320831
:100500008C0033088D008F015A305A20031D8E2A2B
:100510000130AE020030031C013EAF020130B400D6
:100520006400063034020318982AD020B40F902AB1
:10053000B20A0319B30F732AD430AC00AD015C309A
:10054000AE00AF01FF285C30A800A901D430AA009A
:10055000AB01D430AC00AD015C30AE00AF01013076
:10056000B200B30132088C0033088D008F0178305F
:100570005A20031DE42AA80A0319A90A0130AC0273
:100580000030031C013EAD0232088C0033088D00A0
:100590008F011E305D20031DD62A0130AA020030D3
:1005A000031C013EAB02AE0A0319AF0A0130B400CE
:1005B0006400063034020318E02AD020B40FD82A91
:1005C000B20A0319B30FB22AFF280130B200B301F7
:1005D00032088C0033088D008F0178305A20031DBB
:1005E0001A2B0130A8020030031C013EA902AC0AFC
:1005F0000319AD0A32088C0033088D008F015A3080
:100600005A20031D0C2BAA0A0319AB0A0130AE02B3
:100610000030031C013EAF020130B400640006301C
:1006200034020318162BD020B40F0E2BB20A031974
:10063000B30FE82A5C30A800A901D430AA00AB01AE
:10064000D430AC00AD015C30AE00AF01FF2801300A
:10065000B200B30132088C0033088D008F0178306E
:100660005A20031D652B0130A8020030031C013EF7
:10067000A9020130AC020030031C013EAD02320879
:100680008C0033088D008F011E305D20031D4B2B25
:10069000AA0A0319AB0A32088C0033088D008F01B7
:1006A0005A305A20031D572BAE0A0319AF0A0130E6
:1006B000B4006400063034020318612BD020B40F5C
:1006C000592BB20A0319B30F2A2B5C30A800A901D9
:1006D000D430AA00AB01FF280130B200B3013208C8
:1006E0008C0033088D008F0178305A20031DAA2B0F
:1006F000A80A0319A90AAC0A0319AD0A32088C002A
:1007000033088D008F011E305D20031D8D2B0130BD
:10071000AA020030031C013EAB0232088C003308F1
:100720008D008F015A305A20031D9C2B0130AE02E0
:100730000030031C013EAF020130B40064000630FB
:1007400034020318A62BD020B40F9E2BB20A031933
:10075000B30F6F2BD430AC00AD015C30AE00AF01F5
:10076000FF285C30A800A901D430AA00AB01D43026
:10077000AC00AD015C30AE00AF010130B4006400EC
:10078000C93034020318C72BD020B40FBF2BFF2869
:040790006300C82B0F
:02400E00F13F80
:00000001FF
